:10000000560A28001402B402240008022000520AF2
:100010002E004E090E022C000A066C00160943063B
:10002000520A16094306520A1609520A0E02AC0178
:10003000010C2A006B0000024E018C0143070008EE
:10004000AA024306EB031B0A000824006000A40276
:100050008406260A520A6D002C00FF0CEC010307EF
:10006000ED010307520A030C2B00DF0C39092D0A9E
:100070006B002A00E70CEA016B02FC0C0307440A40
:10008000EA010306400AEA010000EB03400A0A06FF
:10009000490A2A074D0A00004D0A000807012700F7
:1000A0000600520AC404A404000000086400FF0C07
:1000B00027002900100C3400A90409020200100CCA
:1000C0002509470507020600010C3600040C9600BE
:1000D0000306780A2605270407020600C80C2B0928
:1000E0002604270407020600C80C2B09F603660A3B
:1000F000010C2A00060C2400080C08090A0235002D
:100100000F0C2B09320C95000306870A640A1702AC
:100110004306010C430740002F004C0C95004000A3
:100120000306010C4F012F007D0C9500010C030606
:1001300040004F0143069E0A010C3700010C970056
:100140004306010C430740002F00B00C950040000F
:100150000306010C4F012F00E10C9500010C030672
:1001600040004F014306B60A020C3700020C97000C
:100170004306010C430740002F004C0C9500400043
:100180000306010C4F012F007D0C9500010C0306A6
:1001900040004F014306CE0A030C3700030C9700C2
:1001A0004306010C430740002F00B00C95004000AF
:1001B0000306010C4F012F00E10C9500010C030612
:1001C00040004F014306E50AFE0A040C970043066F
:1001D000010C430740002F004C0C95004000030623
:1001E000010C4F012F007D0C9500010C030640000F
:1001F0004F014306FD0A030C3700780A4606030B3D
:10020000010C01091B0B8604870407020600260562
:10021000270407020600FA0C2B09870507020600CF
:100220002604270407020600040C37000B0C2D00DF
:10023000B80C2C09780AA604A70407020600010CD2
:100240002D00F40C2C09A70507020600010C2D0057
:10025000F40C2C09D400F4002400000228006400EF
:02026000FC0B95
:0803F800E802F90B030B000001
:021FFE00EA0FE8
:00000001FF
